:100000000C9462000C94E41B0C94111C0C948A0058
:100010000C948A000C948A000C948A000C948A0038
:100020000C948A000C948A000C948A000C948A0028
:100030000C948A000C9430070C948A000C948A006B
:100040000C943E1C0C948A000C949F1F0C94DA1F95
:100050000C948A000C948A000C948A000C948A00F8
:100060000C94B4050C948A000000000024002700C2
:100070002A0000000000250028002B0000000000DE
:1000800023002600290004040404040404040202DA
:100090000202020203030303030301020408102007
:1000A0004080010204081020010204081020000012
:1000B0000007000201000003040600000000000029
:1000C0000000932111241FBECFEFD8E0DEBFCDBFCB
:1000D00012E0A0E0B1E0EEEBF4E402C005900D9276
:1000E000A23DB107D9F714E0A2EDB2E001C01D9224
:1000F000AB3BB107E1F710E0C4ECD0E004C02297BD
:10010000FE010E945922C23CD107C9F70E94D821A2
:100110000C945D220C940000FB01DC0102C00190F4
:100120000D9241505040D8F708958091D20281300D
:1001300019F482E08093D2028091D202833019F4C4
:1001400084E08093D202089520E030E040E050E067
:1001500060E071E0F999FECF72BD61BDF89A80B59B
:10016000542F432F322F2227280F311D411D511D9F
:100170006F5F7F4F81E06430780761F72E513E4B0F
:10018000414C5E4D19F020E030E01AC024E031E02F
:10019000F999FECF32BD21BDF89A80B5F901E1533E
:1001A000FE4F80832F5F3F4F81E02D32380781F76C
:1001B00020E030E08091D302893011F421E030E07A
:1001C000C90108958436910520F4BC0180E090E0D7
:1001D00025C08E3B910550F48A559040BC0180E0CB
:1001E00090E02AE030E040E050E016C0823D91050A
:1001F00050F4845B9040BC0180E090E024E630E065
:1002000040E050E009C08D5C9040BC0180E090E08F
:1002100028E532E040E050E00E94E72124E630E0AB
:1002200040E050E00E94E721089590E08C599F4FF4
:100230000E94E2000895DC019896EC91F0E0E770EE
:10024000F070E654FD4F80810895FC0120A530E058
:10025000C90181709070019627703070359527958F
:10026000820F931F880F880F08958F929F92AF92ED
:10027000BF92CF92DF92EF92FF920F931F938C0168
:100280000E941B01D80197962C9130E043E150E089
:10029000249FF001259FF00D349FF00D1124EE5F97
:1002A000FD4F80809180A280B38090E00F96AA27B6
:1002B00097FDA095BA2FBC01CD0120E43FE14DE7A9
:1002C00050E00E94E721A50194010E941A226901D1
:1002D0007A0180ED97E0A0E0B0E0C80ED91EEA1EDA
:1002E000FB1ED80198968C91887181F060E07EEEBB
:1002F0008AEB9BE0A50194010E941A2228513C4FF1
:100300004F4F5F4FC20ED31EE41EF51E87EE93E0E3
:10031000A0E0B0E0C80ED91EEA1EFB1EC701B60160
:1003200028EE33E040E050E00E941A22CA01B901F1
:1003300028EE33E040E050E00E94E7211F910F914A
:10034000FF90EF90DF90CF90BF90AF909F908F90F5
:1003500008958F3F910509F010F480E0089522E0A0
:100360008030920710F481E008958050934010F09F
:1003700083E0089582E00895CF92DF92FF920F9379
:100380001F93CF93DF93F82FEB016A01182F169577
:10039000E0E088819981D6018C938A819B811196B6
:1003A0008C9311978C819D8112968C9312978E81DC
:1003B0009F8113968C931397288139814A815B81A1
:1003C0006C817D818E819F819295990F990F907C90
:1003D000832F8370982B852F8370880F880F982B1D
:1003E000872F83708295807F982B14969C9385E04D
:1003F00090E0C80ED91E2896EF5F1E1750F6F0FF4A
:1004000021C0888199810E94A901F82E8A819B814F
:100410000E94A901182F8C819D810E94A901082F9B
:100420008E819F810E94A901F294FF0CFF0C50EC79
:10043000F5221295107F1F29182B000F000F012B9A
:10044000D6010C93DF91CF911F910F91FF90DF9018
:10045000CF9008951F93182FDB01FA01482F46957E
:1004600030E0848190E083709070982F88272081FD
:10047000820F911D11969C938E93848190E08C70D5
:10048000907066E0880F991F6A95E1F72181820FCD
:10049000911D13969C938E931297848190E08073A4
:1004A000907054E0880F991F5A95E1F72281820FCE
:1004B000911D15969C938E931497848190E0807C77
:1004C0009070880F991F880F991F2381820F911DAB
:1004D00017969C938E931697359618963F5F431701
:1004E00008F0BFCF10FF50C0808182958695869519
:1004F000837090E02DE431E0AC01429FC001439F46
:10050000900D529F900D11240C9611969C938E93F2
:10051000808190E074E0969587957A95E1F78370F5
:100520009070AC01429FC001439F900D529F900D6F
:1005300011240C9613969C938E931297808190E0D1
:10054000969587959695879583709070AC01429F9C
:10055000C001439F900D529F900D11240C9615964B
:100560009C938E931497808190E083709070AC017F
:10057000429FC001439F900D529F900D11240C96F5
:1005800017969C938E9316971F9108958C30910522
:1005900048F49C01B4E0220F331FBA95E1F7285DBF
:1005A0003C4F17C023E0843F920720F49C01245263
:1005B0003C4F0FC024E08030920718F020E938E06B
:1005C00008C09C012657334FA4E0220F331FAA9581
:1005D000E1F7C90108959C01369527952575357574
:1005E000821B930B9C01369527953695279523738F
:1005F000337383739373280F391FC90144E09695B1
:1006000087954A95E1F7820F931F8F709F7021E0C5
:1006100031E0AC01429FC001439F900D529F900D6D
:100620001124892F0895382F20E0809102049091A1
:1006300003048227932740E061E270E19C01220FCE
:10064000331F97FF04C0C9018627972701C0C9013E
:100650004F5F483099F79093030480930204089504
:10066000882339F02D9800002B9A00002D9A000065
:1006700008952D9800002B9800002D9A00000895F1
:100680002D9A000083B12D98000090E0F4E096953B
:100690008795FA95E1F7817008950F931F93082FBE
:1006A0005C9A2D985C9810E0802F80780E9430032F
:1006B000000F1F5F1830C1F72D981F910F910895FB
:1006C0008F770E944D0308950F931F93082F10E01A
:1006D000802F80780E943003000F1F5F1830C1F711
:1006E0002D981F910F9108950F931F932D9880E0DF
:1006F00000E0182F110F0E944003810F0F5F083098
:10070000C1F71F910F9108950E9460030E94740326
:100710005C9A08951F93162F80680E944D03812FC5
:100720000E9464035C9A1F9108951F931091DC024C
:100730001827E3EDF2E0E80FF11D89E767850E94D5
:100740008A038DE3612F0E948A0382E4612F0E9455
:100750008A031F91089586E20E94840308950F93EF
:100760001F938BE20E948403082F8CE20E94840373
:10077000282F30E0B6E036952795BA95E1F710E0DE
:10078000000F111F000F111F202B312BC9011F91CA
:100790000F9108950F931F938C018CE1F8016481F0
:1007A0000E948A038DE1F80165810E948A038EE12F
:1007B000F80166810E948A0380E2F80167810E9445
:1007C0008A0381E2F80160850E948A0382E2F801CF
:1007D00061850E948A0383E2F80162850E948A0390
:1007E00084E2F80163850E948A0385E2F80164854A
:1007F0000E948A038AE2F80165850E948A038EE6D8
:10080000F80166850E948A038FE6F80167850E94D9
:100810008A0380E7F80160890E948A0381E7F80172
:1008200061890E948A0382E7F80162890E948A0333
:100830001F910F910895EF92FF920F931F93CF9303
:10084000DF937B018C01603028E372072CE982077B
:100850002CE1920728F520E836E948E950E00E94AB
:100860001A22E9016897B90180E090E020E839E6B2
:1008700047E65FEF0E94E7216E0D7F1D801F911FED
:1008800002E0660F771F881F991F0A95D1F721E7AD
:1008900032E040E050E00E941A22890180E421C049
:1008A00020E03DE241E351E00E941A22E90168970D
:1008B000B90180E090E020E033ED4EEC5EEF0E9465
:1008C000E7216E0D7F1D801F911F660F771F881F08
:1008D000991F21E732E040E050E00E941A2289018E
:1008E00080E69E012F71622F680F85E70E948A03C0
:1008F00086E7612F0E948A0387E7602F0E948A03A0
:10090000DF91CF911F910F91FF90EF9008959F92EB
:10091000AF92BF92CF92DF920F93DF93CF9300D02D
:1009200000D0CDB7DEB7982E83E00E948403809379
:10093000170384E00E9484038093180386E060E03C
:100940000E948A0387E061E00E948A0389E06FE7E2
:100950000E948A038AE065E00E948A038BE062E1DC
:100960000E948A038CE065E10E948A038DE06DEFAE
:100970000E948A038EE060E00E948A03992019F0A9
:1009800081E692E008C08091FA0223E1829FC001D3
:1009900011248E5F9D4F0E94CA0380E36CE80E9481
:1009A0008A0382E36FE00E948A0383E362E40E9489
:1009B0008A0384E36AE00E948A0385E36AE20E9474
:1009C0008A0386E36DE20E948A0387E364ED0E9456
:1009D0008A0388E360E00E948A0389E360E00E9462
:1009E0008A03992049F02EE1A22E2EEBB22E21ECA3
:1009F000C22E2EEDD22E08C0A090DC02B090DD02F7
:100A0000C090DE02D090DF020AE38D2D9927AA273D
:100A1000BB2789839A83AB83BC83802F69810E9423
:100A20008A03802F8B5F69810E948A03DC2CCB2C88
:100A3000BA2CAA240F5F0E3341F783E46FEF0E94B4
:100A40008A0384E46FEF0E948A0385E46FEF0E94BB
:100A50008A0386E46FEF0E948A03992019F08DE6DD
:100A600066E003C08DE66091E0020E948A0389E798
:100A700060E00E948A038AE76091E1020E948A0393
:100A800083E760E00E948A0384E760E00E948A03B3
:100A9000992029F060EC72E98DEE99E108C060912F
:100AA000D8027091D9028091DA029091DB020E9403
:100AB0001B040F900F900F900F90CF91DF910F912B
:100AC000DF90CF90BF90AF909F90089587E061E056
:100AD0000E948A038EE764E20E948A0388E063E052
:100AE0000E948A0388E060E00E948A0387E065E054
:100AF0000E948A0385E062E00E948A0383E00E94EC
:100B000084038093170384E00E9484038093180376
:100B1000089590E0411191E0880F982B9093BA00CE
:100B2000660F6093BD0030931E0320931D0308954C
:100B3000882311F085EC01C085E88093BC000895FE
:100B400085ED8093BC008091BC0084FDFCCF0895AE
:100B500085EC8093BC000895ECEBF0E0108285E416
:100B600080831092230308951F920F920FB60F9265
:100B700011242F933F934F935F936F937F938F93A2
:100B80009F93AF93BF93EF93FF93DF93CF930F9216
:100B9000CDB7DEB78091B90090E0887F9070803645
:100BA000910509F4EAC081369105CCF588329105AA
:100BB00009F47CC089329105B4F48031910509F4BF
:100BC00070C0813191053CF4009709F40EC108977B
:100BD00009F00DC166C08831910509F467C080979E
:100BE00009F005C177C08034910509F490C08134C3
:100BF000910544F48033910509F46EC0C89709F05B
:100C0000F6C06CC08035910509F471C08835910536
:100C100009F483C08834910509F0E9C0A5C088397A
:100C2000910509F4DCC089399105ECF48837910508
:100C300009F4A3C0893791054CF48836910509F46D
:100C40009CC08037910509F0D2C097C088389105C3
:100C500009F4C5C08039910509F492C08038910526
:100C600009F0C5C08DC0803B910509F4A5C0813B4A
:100C700091054CF4803A910509F499C0883A9105A0
:100C800009F0B5C099C0803C910509F4AAC0883C20
:100C9000910509F4A6C0883B910509F0A8C080E041
:100CA0008CC080911F038093BB009BC08091220366
:100CB0008150809322038F5F09F43FC0E0912003AD
:100CC000F091210381918093BB00F0932103E09385
:100CD000200387C082E049C083E047C084E080935E
:100CE0002403809123038B7F8093230362C0809130
:100CF000BB00E0912003F09121038193F093210345
:100D0000E0932003809122038150809322038091FD
:100D10002203823008F065C062C08091BB00E09180
:100D20002003F09121038193F0932103E0932003AA
:100D300080912203815080932203809123038B7F33
:100D4000809323038091230380FF4FC0809123036E
:100D50008E7F8093230380912303826080932303FB
:100D600084EA8093BC0043C085E080932403809193
:100D700023038B7F8093230338C01092220331C05A
:100D8000E0911D03F0911E03309749F19091BB0053
:100D9000809122038F5F80932203815011F060E0E5
:100DA00001C062E09983CE01019609951BC00E94A3
:100DB000A0050E94A8051BC081E0E0911D03F091F1
:100DC0001E03309761F0882311F461E001C063E0F5
:100DD000CE010196099599819093BB0003C080E0F4
:100DE00001C081E00E94980502C00E94A0050F90FA
:100DF000CF91DF91FF91EF91BF91AF919F918F9133
:100E00007F916F915F914F913F912F910F900FBE06
:100E10000F901F90189525B190E0FC01EE0FFF1F79
:100E2000E80FF91FE657FC4F8081282B25B988B1C0
:100E30009181892B88B98BB19281892B8BB90895C7
:100E400085B19091BA03892385B988B19091BB038C
:100E5000892388B98BB19091BC0389238BB90895FC
:100E60001F920F920FB60F9211241F932F933F934F
:100E70004F935F936F937F938F939F93AF93BF93A2
:100E8000CF93DF93EF93FF9310915C0380919802CF
:100E9000C0919602D0919702181708F05BC080911C
:100EA000BD039091BE039093870080938600E12F4D
:100EB000F0E0EE0FFF1FEC58FD4F808191810E9402
:100EC000C602880F991F9093BE038093BD03809143
:100ED000BD039091BE039E01281B390BC9013093BD
:100EE0009702209396022091120330911303220F50
:100EF000331F8217930720F43093970220939602B2
:100F000080915E03882339F480910A0380FF59C0E1
:100F1000183008F456C08FEF9FEF909389008093AC
:100F2000880080918400909185008097D0F30E9482
:100F3000200780915D03882339F480915C03882326
:100F400019F081500E940B0780915C038F5F8093A2
:100F50005C033EC08091BD039091BE0390938700D7
:100F600080938600D093BE03C093BD0380915E033F
:100F7000882319F08FEF9FEF06C08091BD039091F9
:100F8000BE0388559240909389008093880080E446
:100F90009CE99093970280939602809184009091AF
:100FA00085008097D0F30E94200780915D038823FD
:100FB00029F48091980281500E940B0710925C03E3
:100FC00007C08091BD039091BE0388559240A5CF84
:100FD000FF91EF91DF91CF91BF91AF919F918F9151
:100FE0007F916F915F914F913F912F911F910F9042
:100FF0000FBE0F901F90189590E0880F991F880FD3
:10100000991F8C30910518F42CE030E007C09C014A
:1010100083E0253F380710F024EF33E0C90108953D
:10102000DF93CF93CDB7DEB764970FB6F894DEBFEA
:101030000FBECDBF20E030E0AE014F5F5F4FF999AA
:10104000FECF20583E4F32BD21BD20583140F89A86
:1010500080B5FA01E20FF31F80832F5F3F4F2430EA
:10106000310569F789818A3F51F58A81813139F5E6
:101070008B818A3521F58C818E3F09F520E030E0A7
:10108000AE014F5F5F4FF999FECF2C573E4F32BDF7
:1010900021BD24583140F89A80B5FA01E20FF31FC0
:1010A00080832F5F3F4F2431310569F786E060E68A
:1010B00073E00E942A0281E08093800302C01092B4
:1010C000800364960FB6F894DEBF0FBECDBFCF91FC
:1010D000DF910895809180038823E9F080910B03CC
:1010E000482F50E0A0E6B3E020E030E024173507B9
:1010F00061F0F8948D919C911197F901EE0FFF1F0B
:10110000EC58FD4F9183808378942F5F3F4F129668
:101110002031310559F708951F93CF93DF93EC01E8
:1011200070E0CB018270907060FF1AC0892B31F0A3
:101130008091830388831092010445C010910104BB
:1011400083ED92E00E941B011817D8F5E12FF0E023
:10115000E154FC4F808188831F5F1093010433C0EA
:10116000892BC1F098819093000410920104892F7B
:10117000807E803651F480918303823010F1888123
:101180008F718093410383E01AC09E3FE1F4109277
:10119000830317C0809100048F3FA9F420910104BC
:1011A000293278F4E22FF0E0ED52FD4F8881808300
:1011B000822F8F5F80930104893229F481E080932C
:1011C000830380E001C081E0DF91CF911F910895FA
:1011D000EF92FF920F931F93CF93DF9380E260E033
:1011E00040E02CE838E00E94890510928303E2E099
:1011F000EE2E75E0F72E04E080918303813039F400
:1012000080E00E948704E09283035E98F5CF1091FE
:101210008303133061F45D98809141030E9495032C
:101220001093D2020E94660500938303E5CF80915C
:101230008303843009F78091D2028430E9F68FE786
:101240000E946003C0E0D0E007C00E947403FE016A
:10125000E154FC4F8083219683ED92E00E941B01B4
:1012600090E0C817D9078CF3F09283035D9AC4CF3E
:10127000AF92BF92CF92DF92EF92FF920F931F93A4
:10128000CF93DF93EC010E94941C5B016C017E0103
:1012900000E010E011C0209779F00E94941C6A19B8
:1012A0007B098C099D09E616F7060807190720F443
:1012B0000E94AC0581E008C08091230382FDEBCF42
:1012C0008091240310922403DF91CF911F910F91FD
:1012D000FF90EF90DF90CF90BF90AF900895CF92A6
:1012E000DF92EF92FF920F931F93CF93DF93182F0C
:1012F0007B01042FC22FD0E0F4E0CF2ED12CCC22E2
:10130000DD2222FF03C080E090E004C080919402BF
:10131000909195020E943809282F8823B1F51092E8
:10132000240300932203F0922103E0922003110F83
:10133000116010931F0390912303C1FD02C084E04C
:1013400001C085E0892B809323038091230381FFD3
:101350000BC0809123038D7F8093230380911F0313
:101360008093BB0085EC01C085EE8093BC00C0FF7C
:101370000CC0CD2819F080E090E004C08091940268
:10138000909195020E943809282F822FDF91CF91EA
:101390001F910F91FF90EF90DF90CF900895CF9223
:1013A000DF92EF92FF920F931F93CF93DF93182F4B
:1013B0007B01042FC22FD0E0A4E0CA2ED12CCC2276
:1013C000DD2222FF03C080E090E004C080919402FF
:1013D000909195020E943809282F8823A9F5109230
:1013E000240300932203F0922103E0922003110FC3
:1013F00010931F0390912303C1FD02C084E001C03C
:1014000085E0892B809323038091230381FF0BC008
:10141000809123038D7F8093230380911F0380930A
:10142000BB0085EC01C085EE8093BC00C0FF0CC002
:10143000CD2819F080E090E004C080919402909152
:1014400095020E943809282F822FDF91CF911F919A
:101450000F91FF90EF90DF90CF9008958091D2028E
:10146000813011F081E008950E94941C20911903AD
:1014700030911A0340911B0350911C03621B730BA4
:10148000840B950B615A76488140904010F480E0BF
:10149000089582E00895FF920F931F93CF93DF93F7
:1014A000182F092FF62E8EE30E948A03212F302F4A
:1014B000C901EC0110E005C08FE769910E948A0321
:1014C0001F5F1F15C8F385E064E00E948A0383E074
:1014D0000E9484038093170384E00E948403809316
:1014E00018030E94941C6093190370931A0380934D
:1014F0001B0390931C0387E069E00E948A0381E04C
:101500008093D202DF91CF911F910F91FF900895A8
:101510000E944B0A8091D2028130D9F40E94941C1F
:101520002091190330911A0340911B0350911C0321
:10153000621B730B840B950B605A76488140904078
:1015400040F4E8CF89E994E060E071E00E948A1FEE
:1015500008958091D2028130A9F30895DF93CF934B
:101560000F92CDB7DEB7809183038230B9F480E269
:10157000BE016F5F7F4F41E021E00E946F09882329
:1015800079F08FEF809383030E94861C609384031D
:101590007093850380938603909387038FEF01C038
:1015A00089810F90CF91DF910895DF93CF930F92B0
:1015B000CDB7DEB7809183038230D9F480914103A7
:1015C000805A898380E2BE016F5F7F4F41E021E056
:1015D0000E94CF09882369F08FEF809383030E94D4
:1015E000861C609384037093850380938603909395
:1015F00087030F90CF91DF9108950F931F93DF938F
:10160000CF93CDB7DEB7AA970FB6F894DEBF0FBE63
:10161000CDBF8FEF8983DE011296E3EDF2E089E220
:1016200001900D928150E1F780E28E010F5F1F4F14
:10163000B8014AE221E00E94CF09882351F480E2F8
:10164000B80141E021E00E946F09882311F482E093
:1016500001C08FEF8093830380918303823051F028
:101660000E94861C60938403709385038093860395
:1016700090938703AA960FB6F894DEBF0FBECDBF36
:10168000CF91DF911F910F910895EF92FF920F93E9
:101690001F93DF93CF9300D0CDB7DEB70E94941C89
:1016A0009B01AC018091250390912603A091270313
:1016B000B091280379018A01E81AF90A0A0B1B0B79
:1016C000D801C70181519742A040B04008F444C0FE
:1016D000809129038F5F80932903815080FD02C090
:1016E00000E001C007E020932503309326034093D8
:1016F00027035093280389E994E063E00E94532173
:1017000089E994E061E00E94532137E0F32EF00E66
:10171000802F90E0880F991F9C012C583D4F3A83F1
:101720002983F90160817181672F77276370707059
:10173000880F991F682B792B89E994E00E94532127
:10174000E981FA8160817181707089E994E00E9479
:1017500053210F5F0F15E1F60F900F90CF91DF919E
:101760001F910F91FF90EF9008951F93182F89E913
:1017700094E0612F0E945321812F0E9413031F9137
:101780000895CF92DF92EF92FF920F931F93CF9322
:10179000DF93082F0E94941C9B01AC0180912503CC
:1017A00090912603A0912703B091280369017A0143
:1017B000C81AD90AEA0AFB0AD701C6018151974221
:1017C000A040B04008F443C0209325033093260383
:1017D00040932703509328031092030410920204AD
:1017E00088EA0E94B50B002311F481E001C081E872
:1017F0000E94B50B80E10E94B50BC0E0D0E0FE0175
:10180000EE0FFF1FEC58FD4F808191810E94C602B0
:101810008C0143E0000F111F4A95E1F7812F0E94D0
:10182000B50B802F0E94B50B2196C031D10539F739
:101830006091030489E994E00E94532160910204BD
:1018400070910304707089E994E00E945321DF9144
:10185000CF911F910F91FF90EF90DF90CF9008955F
:10186000CF92DF92EF92FF920F931F93CF93DF936C
:10187000182F062F0E94941C9B01AC018091250318
:1018800090912603A0912703B091280369017A0162
:10189000C81AD90AEA0AFB0AD701C6018151974240
:1018A000A040B04008F4D6C120932503309326030E
:1018B00040932703509328038091740290917502FE
:1018C000880F991F80932A03977080912B03887F3C
:1018D000892B80932B032091760230917702220F7F
:1018E000331F922F990F990F990F8770892B80932F
:1018F0002B03422F42954695477080912C03807CA4
:10190000932F9770990F990F990F842B892B8093A0
:101910002C032091780230917902220F331F922FED
:101920009295990F990F907C8F73892B80932C033C
:10193000932F9295990F990F907C822F869586957B
:10194000892B80932D03932F969596959170809176
:101950002E038E7F892B80932E0320917A02309163
:101960007B02220F331F922F990F8170892B809356
:101970002E03422F441F4427441F80912F03807F52
:10198000932F9770990F842B892B80932F0320918D
:101990007C0230917D02220F331F922F9295907F0F
:1019A0008F70892B80932F03422F42954F70809127
:1019B00030038078932F97709295907F842B892B9A
:1019C0008093300320917E0230917F02220F331FDB
:1019D0008F7780933003932F979599279795822F30
:1019E0008695892B80933103932F969593708091E0
:1019F00032038C7F892B8093320340918002509177
:101A00008102440F551F942F990F990F8370892BD2
:101A100080933203942F929596959695937020918A
:101A20003303207E852F8770880F880F292B282B62
:101A3000209333038091820290918302880F991F33
:101A4000382F3295330F307E2F71232B20933303A1
:101A5000292F2295220F207E869586958695822BAA
:101A6000809334038091840290918502880F991F9E
:101A700080933503977080913603887F892B8093FC
:101A800036032091860230918702220F331F922F56
:101A9000990F990F990F8770892B80933603422FE6
:101AA00042954695477080913703807C932F9770BD
:101AB000990F990F990F842B892B809337032091CD
:101AC000880230918902220F331F922F9295990F2D
:101AD000990F907C8F73892B80933703932F929566
:101AE000990F990F907C822F86958695892B8093EC
:101AF0003803932F969596959170809139038E7F38
:101B0000892B8093390320918A0230918B02220F16
:101B1000331F922F990F8170892B80933903422FA5
:101B2000441F4427441F80913A03807F932F97706E
:101B3000990F842B892B80933A0320918C0230914A
:101B40008D02220F331F922F9295907F8F70892BD9
:101B500080933A03422F42954F7080913B038078E7
:101B6000932F97709295907F842B892B80933B03C2
:101B700020918E0230918F02220F331F8F77809336
:101B80003B03932F979599279795822F8695892BBD
:101B900080933C03932F9695937080913D038C7FA7
:101BA000892B80933D034091900250919102440F04
:101BB000551F942F990F990F8370892B80933D03A4
:101BC000942F929596959695937020913E03207E42
:101BD000852F8770880F880F292B282B20933E0391
:101BE0008091920290919302880F991F382F32951D
:101BF000330F307E2F71232B20933E03292F229504
:101C0000220F207E869586958695822B80933F03B2
:101C1000112311F490E001C098E0002311F480E05A
:101C200001C084E0892B8093400389E994E06FE050
:101C30000E945321CAE2D3E089E994E069910E94AD
:101C4000532183E0C134D807B9F789E994E060E013
:101C50000E945321DF91CF911F910F91FF90EF9040
:101C6000DF90CF900895CF93DF9389E994E00E94AD
:101C7000E020892BF9F08091FE03C82FD0E09E016F
:101C80002F5F3F4F2F7130708091FD0390E0281738
:101C9000390781F089E994E00E941A21C352DC4F90
:101CA00088838091FE0390E001968F7190708093FD
:101CB000FE03DBCFDF91CF9108958CE060E00E94BE
:101CC000251D8BE061E00E94251D8DE061E00E94F2
:101CD000251D82E060E00E94251D84E061E00E94F5
:101CE000251D089583E00E9484038093170384E0F8
:101CF0000E9484038093180387E061E00E948A03B6
:101D00006AE070E080E090E00E94BA1C0E946605E4
:101D1000000008950F931F93082F17C05E9A64E682
:101D200070E080E090E00E94BA1C5E9864E670E08B
:101D300080E090E00E94BA1C1F5F101778F36CE2FD
:101D400071E080E090E00E94BA1C10E0F6CF482FCE
:101D5000392F25E00DC0F999FECF1FBA842F932F9C
:101D600092BD81BD60BD0FB6F894FA9AF99A0FBE84
:101D7000215059F0F999FECF842F932F92BD81BD48
:101D8000F89A80B5681739F7089582E00E948A0EA4
:101D90000895CF92DF92EF92FF920F931F93CF930C
:101DA000DF93C8E1D0E000E411E03EE1C32E3EEB5A
:101DB000D32E31ECE32E3EEDF32EA70196010C2E2F
:101DC00004C056954795379527950A94D2F7C801D0
:101DD000622F0E94A70E28970F5F1F4F8FEFC83FFB
:101DE000D80759F7C4E4D1E0FE01E854FE4FCE0114
:101DF00060810E94A70E219681E0CF35D807A1F718
:101E0000DF91CF911F910F91FF90EF90DF90CF90D6
:101E1000089522E02093FC021092FD0291E090933D
:101E2000FE022093FF0293E09093000394E09093CE
:101E3000010395E09093020394E29093030395E2EB
:101E40009093040320930A039FEF90930B032AE0DF
:101E500020931403109215031092160310920C0392
:101E600010920D0310920E0310920F039EE19093B7
:101E700010032093110328EB3BE0309313032093CE
:101E80001203882311F00E94C90E089520E030E06B
:101E900040E050E060E471E0F999FECF72BD61BDB1
:101EA000F89A80B5542F432F322F2227280F311D47
:101EB000411D511D6F5F7F4F81E06434780761F7EA
:101EC0002E513E4B414C5E4D21F081E00E94090FA6
:101ED000089524E431E0F999FECF32BD21BDF89A8E
:101EE00080B5F901E854FE4F80832F5F3F4F81E0BA
:101EF0002F35380781F78091FC02823019F081E09C
:101F00000E94090F89E994E06CE071E00E948A1F49
:101F100008952F923F924F925F926F927F928F928D
:101F20009F92AF92BF92CF92DF92EF92FF920F9368
:101F30001F93DF93CF93CDB7DEB7C054D0400FB619
:101F4000F894DEBF0FBECDBF6B017C010E94861CE2
:101F50004B015C0181E00E94870483E08093D20200
:101F60000E94720E89E994E06AE171E00E948A1F82
:101F70001E010894211C311CA3E24A2E512C4C0E48
:101F80005D1EFEE16F2E712C6C0E7D1E80C089E9F6
:101F900094E068E271E00E948A1F8FE70E9460036C
:101FA0000E9474038983823601F503ED12E00E94DA
:101FB0007403F80181938F01F2E00C3F1F07B9F71A
:101FC0008091D302893009F05DC089E994E061E332
:101FD00071E00E948A1F82E48983CE01019661E04C
:101FE0000E94880A5D9A81E068C0803719F08936BE
:101FF000C9F406C080E58A83CC24DD24760105C0BF
:1020000081E00E94090FE9E4EA83DE011396ECEF18
:10201000F2E08BE101900D928150E1F7CE01029642
:102020006CE12EC08437C9F4F4E5FE8F83E08F8F16
:10203000F8A3E8E0E9A3FFE0FAA3D201E4EEF1E0BF
:102040008EE101900D928150E1F7C30163E20E949D
:10205000880ACC24DD24760115C0853799F40CEF6D
:1020600012E00E947403F80181938F01F3E00731BD
:102070001F07B9F70E94C90E85E58983C10161E098
:102080000E94880AE3E0E093D2020E946605C11430
:10209000D104E104F10459F00E94861C6819790901
:1020A0008A099B096C157D058E059F0528F4809192
:1020B000D202843061F76BCF80E0C05CDF4F0FB697
:1020C000F894DEBF0FBECDBFCF91DF911F910F916E
:1020D000FF90EF90DF90CF90BF90AF909F908F9048
:1020E0007F906F905F904F903F902F900895CF9288
:1020F000DF92EF92FF920F931F93CF93DF93C8E18C
:10210000D0E000E011E0BEE1CB2EBEEBDB2EB1EC67
:10211000EB2EBEEDFB2EA70196010C2E04C05695AA
:102120004795379527950A94D2F7C801622F0E94E8
:10213000A70E28970F5F1F4F8FEFC83FD80759F79B
:10214000C4E0D1E0FE01E153FE4FCE0160810E9468
:10215000A70E219681E0CD32D807A1F7DF91CF916C
:102160001F910F91FF90EF90DF90CF900895AF9265
:10217000BF92CF92DF92EF92FF920F931F93DF9364
:10218000CF93CDB7DEB764970FB6F894DEBF0FBE1E
:10219000CDBF0E94861C5B016C01A0E6B3E020E08D
:1021A00030E0F901EE0FFF1FEC58FD4F8081918167
:1021B0008D939D932F5F3F4F2031310591F781E043
:1021C0008093800386E060E673E08E010F5F1F4F0F
:1021D000A8010E94BC01EE24FF24F801EE0DFF1DB2
:1021E000C7018C579E4F60810E94A70E0894E11C86
:1021F000F11C84E1E816F10481F78AEF898381E11B
:102200008A838AE58B838EEF8C8300E010E07E0169
:102210000894E11CF11CF701E00FF11FC801805880
:102220009E4F60810E94A70E0F5F1F4F0430110563
:1022300091F70E94861C9B01AC012A193B094C09AD
:102240005D09283C31054105510550F468EC70E00A
:1022500080E090E0621B730B840B950B0E94BA1C0C
:1022600064960FB6F894DEBF0FBECDBFCF91DF915D
:102270001F910F91FF90EF90DF90CF90BF90AF90A4
:1022800008951F93CF93DF93CDEFD2E010E08881C4
:10229000E82FF0E084FF11C0EF70F070EE0FFF1F29
:1022A000EC58FD4F8081918160E08F3F910511F0E6
:1022B00008F061E0812F0E94911D1F5F2196183068
:1022C00031F7DF91CF911F9108951F93182F8091BF
:1022D00002038B3221F485E0612F0E94911D8091D1
:1022E000FF02873259F4112321F08091B000806100
:1022F00003C08091B0008F7E8093B0001F9108953D
:10230000EF92FF921F93CF93DF9383ED92E00E94B1
:1023100025018093980290910B03981719F49F5F01
:1023200090939802EAE8F3E01082118212823396C9
:1023300083E0E23AF807C1F78FEF8093BA03809306
:10234000BB038093BC033DEFE32E32E0F32EA2EA01
:10235000B2E0E7016FEF5FEF4FEF88818031F0F47B
:1023600090E03C91FC01EE0FFF1FE80FF91FE657CC
:10237000FC4F8081832B808311962C911197818152
:10238000822B818312969C9112978281892B828362
:1023900030954323209552239095692321961396D7
:1023A000E3E0C530DE07C9F66093BC035093BB037E
:1023B0004093BA03CAE9D2E010E0F701808182328B
:1023C00038F08632B0F0863219F4888160E00FC0B0
:1023D000163021F48091C1008F7E05C0173029F49A
:1023E0008091C100877F8093C100888161E00E9455
:1023F000251D1F5F0894E11CF11C21961830E9F699
:102400008091FD02803231F489E061E00E94911DEB
:1024100082E801C082E08093800081E080935D03C8
:1024200080935E038091FF02813211F08732D9F4EC
:1024300083E061E00E94251D83E060E00E94911D21
:102440008091FF02813231F481E08093B10080936A
:10245000B00009C082E08093B00085E08093B100B5
:102460008EE38093B3008AE1809381008FEF9FEF2A
:10247000909389008093880080ED97E09093870087
:102480008093860080E49CE9909397028093960263
:102490009093BE038093BD0310925C0380916F0004
:1024A000816080936F0080910A0383FF0AC080914E
:1024B0008003882331F00E946A0810925E03109214
:1024C0005D03DF91CF911F91FF90EF9008950F93DF
:1024D0001F9380915A0390915B039F770E94EB02B8
:1024E000982F8F3031F480915603869586958054CD
:1024F00004C08DE0989FC001112480935703009180
:102500000B03003170F4F89410E0809157030E949F
:10251000FC07000F111F0C581D4FF8019183808399
:1025200078948091FF028132C9F490915703892FEA
:1025300081508E3F60F08091B0008F7D8093B0001D
:1025400060E0911161E083E00E94911D07C09093CB
:10255000B4008091B00080628093B0001F910F9111
:1025600008951F93182F811111E082E1612F0E94BD
:10257000911D83E1612F0E94911D10922203109200
:1025800023038091B9008C6F8093B9008CE0809315
:10259000B80085E48093BC001F910895EF92FF92EC
:1025A0000F931F93CF93DF93EB019C01442737FDDB
:1025B0004095542F60E271EA87E090E00E943C224F
:1025C00089011216130614F001E010E0BE018827FD
:1025D00077FD8095982F20E231EA47E050E00E9495
:1025E000E7219801442737FD4095542F0E943C2253
:1025F0007901C0E0D0E009C02B9AC8010E94E01C1C
:102600002B98C8010E94E01C2196CE15DF05A4F38B
:10261000DF91CF911F910F91FF90EF9008955D9AF8
:1026200083E00E9484038093170384E00E94840364
:102630008093180386E060E00E948A0387E061E0EF
:102640000E948A0389E06FE70E948A038AE065E0BE
:102650000E948A038BE062E10E948A038CE065E1BC
:102660000E948A038DE06DEF0E948A038EE060E095
:102670000E948A0380E76CE20E948A0380E360E0A4
:102680000E948A0389E760E00E948A038AE765E086
:102690000E948A0381E762E10E948A0382E762E086
:1026A0000E948A0383E760E00E948A0384E760E077
:1026B0000E948A0360910C0370910D0380910E03B8
:1026C00090910F030E941B048DE667E00E948A032D
:1026D0006AE070E080E090E00E94BA1C87E069E068
:1026E0000E948A036AE070E080E090E00E94BA1CD9
:1026F00088E891E061E070E00E94CE128DE665E02E
:102700000E948A036AE070E080E090E00E94BA1CB8
:1027100088EB91E061E070E00E94CE128DE664E00B
:102720000E948A036AE070E080E090E00E94BA1C98
:102730008DE591E061E070E00E94CE128DE662E0EE
:102740000E948A036AE070E080E090E00E94BA1C78
:102750008FEA90E061E070E00E94CE128DE660E0CA
:102760000E948A036AE070E080E090E00E94BA1C58
:1027700085E091E062E070E00E94CE1287E061E0C7
:102780000E948A035D9808954F925F926F927F92A4
:102790008F929F92AF92BF92CF92DF92EF92FF9271
:1027A0000F931F93DF93CF93CDB7DEB766970FB626
:1027B000F894DEBF0FBECDBF8CE00E948403882357
:1027C00059F489E994E06CE371E00E948A1F80E08B
:1027D0000E9487040E94720E0E94330E0E94941C75
:1027E0000E94AE0AB82E8E010F5F1F4FAA24AA9432
:1027F0008091D202843029F0B5E0EB2EBE1409F0AE
:1028000066C10E94941C6B017C018091D2028430CD
:10281000E9F48FE70E94600300E010E008C00E9426
:102820007403F801E154FC4F80830F5F1F4F83ED69
:1028300092E00E941B0190E00817190784F30E94A0
:10284000AF03909359038093580328C083ED92E01F
:102850000E941B01482F4F5F80E2B80121E00E94D7
:102860006F09882369F0A09283030E94861C6093FD
:102870008403709385038093860390938703B8CF76
:1028800083ED92E00E941B01482F2FEB33E0FE0105
:102890003296C901BF0150E00E948C00C0924203F1
:1028A000D0924303E0924403F092450310928203D6
:1028B00080915A0390915B03880F991F81609093D8
:1028C0005B0380935A035E985D9A80E00E946511D5
:1028D0008091BF03282F30E0C9018E739070892B3F
:1028E00071F5F8948091FB02877064E772E040EC28
:1028F00053E00E942A0200910B03003160F410E0C3
:10290000809157030E94FC07000F111F0C581D4FA8
:10291000F8019183808378948091BF03909189031B
:1029200080FF08C0992399F50E94B71081E0809339
:1029300089032DC0992359F11092890328C0C90138
:1029400088739070C89719F54091D403842F82271B
:1029500087FF1DC040584093D40380910403853203
:10296000B1F410E00AC01F5FE12FF0E0E154FC4F2A
:1029700089E994E060810E945321212F30E0809109
:10298000BF0390E0877090708217930764F780917F
:102990008103882319F481E08093810310925F03FF
:1029A00010925D0310925E038091FB02887109F41E
:1029B00085C04091D4038091BF0390E0242F30E084
:1029C0008227932786FD6CC0407C80E44827409393
:1029D000D4039091FD038091FE03981701F1A5EDBA
:1029E000B3E030E00FC03F5F892F90E0FC01E3527D
:1029F000FC4F20812D9301968F7190708093FD0381
:102A0000383031F09091FD038091FE03981759F70B
:102A1000395C8091D403382B3093D40341C080912A
:102A200055038093D5038091FE02863211F482E132
:102A300005C080910103863251F48EE00E94F41D9E
:102A400095958795959587958093D60302C01092AA
:102A5000D60380910003863211F483E105C0809192
:102A60000203863251F48FE00E94F41D95958795FC
:102A7000959587958093D70302C01092D7038091D4
:102A800059038093D803809158038093D903809190
:102A90005A0390915B039F770E94EB028093DA03C5
:102AA00084ED93E069E00E944B0A02C00E94330E5D
:102AB0000E942E0A8823D1F30E94411183E0809363
:102AC000D2020E94660581E0809388035D980E948F
:102AD000941C5B016C010E94861C2B013C018091BF
:102AE0008203823008F065C0E0904203F090430317
:102AF0000091440310914503809146039091470350
:102B0000A0914803B09149038E159F05A007B10716
:102B100009F44FC083ED92E00E943501A6019501B2
:102B20002E193F09400B510B6C5D75408040904061
:102B30006217730784079507E0F5E0924603F09269
:102B4000470300934803109349030E94AB0380930B
:102B500055032091530330915403280F311D3093B6
:102B6000540320935303609152036F5F60935203A9
:102B70006930F8F0C90170E00E940622CB01709321
:102B80005403609353032091560343E0249F900124
:102B90001124820F931F969587959695879580931C
:102BA00056030E946712109254031092530310921E
:102BB0005203809181039090FF03882309F457C149
:102BC00080908203891408F0D5C183ED92E00E94C1
:102BD00035012091420330914303409144035091C9
:102BE0004503A21AB30AC40AD50A68517C4F8F4F15
:102BF0009F4F6A157B058C059D0508F075C0809177
:102C00005A0390915B03880F991F90935B03809305
:102C10005A0381E080938803882081F440924A031C
:102C200050924B0360924C0370924D0310924E03EE
:102C300010924F031092500310925103809182031F
:102C40008F5F8093820383ED92E00E943501209193
:102C50004203309143034091440350914503260FB2
:102C6000371F481F591F209342033093430340935B
:102C700044035093450381E0809388035E9A0E9449
:102C800065110E94671230C083ED92E00E94350109
:102C90009B01AC018091420390914303A0914403B6
:102CA000B091450386017501E81AF90A0A0B1B0B5E
:102CB000682D70E080E090E00E94E7216E157F05AE
:102CC0008007910788F410925B0310925A0381E009
:102CD000809388030E946712A0924203B09243033C
:102CE000C0924403D092450380918203882309F463
:102CF000E8C090911403992389F180915F038823A0
:102D000069F5892F90E00E94E20020914A033091FA
:102D10004B0340914C0350914D0383017201E21A21
:102D2000F30A040B150B6E157F0580079107B0F4AD
:102D300081E080935F030E946A08809110030E94E3
:102D40001501640D751D861D971D616060934E030E
:102D500070934F0380935003909351039091160307
:102D60009923F1F080915D038823D1F4892F90E0BD
:102D70000E94E20020914A0330914B0340914C03A2
:102D800050914D0383017201E21AF30A040B150BF3
:102D90006E157F058007910718F481E080935D032D
:102DA000909115039923F1F080915E038823D1F46B
:102DB000892F90E00E94E20020914A0330914B035A
:102DC00040914C0350914D0383017201E21AF30AC2
:102DD000040B150B6E157F058007910718F481E031
:102DE00080935E0380910C0390910D03A0910E03DC
:102DF000B0910F030097A105B10509F462C080915D
:102E00004E0390914F03A0915003B091510300974E
:102E1000A105B10509F455C083017201E81AF90A48
:102E20000A0B1B0B17FD4DC06091110370E080E091
:102E300090E028EE33E040E050E00E94E7216E157C
:102E40007F0580079107E8F50E940F1380E00E943C
:102E500087040E9466050E94861C616060934E0391
:102E600070934F0380935003909351032AC083EDD6
:102E700092E00E9435019B01AC0180914203909148
:102E80004303A0914403B091450386017501E81AFC
:102E9000F90A0A0B1B0B692D70E080E090E00E949C
:102EA000E7216E157F058007910758F4A092420331
:102EB000B0924303C0924403D092450381E08093D3
:102EC000880380915E038823B1F4809104038832E3
:102ED00019F40E94450B0FC0893239F480915F03C9
:102EE000609182030E94300C06C08A3221F48091E6
:102EF0005F030E94C10B809188038130B9F4E09197
:102F00004103EF5FE0934103E83131F0F0E0ED522F
:102F1000FD4F8785882311F410924103809141036E
:102F20000E9495030E94D50A109288038091830322
:102F30008F3F21F50E94861C2091840330918503E8
:102F40004091860350918703621B730B840B950B92
:102F5000695E73408040904088F00E94861C6093B8
:102F600084037093850380938603909387030E9464
:102F7000FD0A04C0891409F0B7CE86CE66960FB656
:102F8000F894DEBF0FBECDBFCF91DF911F910F919F
:102F9000FF90EF90DF90CF90BF90AF909F908F9079
:102FA0007F906F905F904F900895FF920F931F93C3
:102FB000082FF62E61E00E94251D802F61E00E94FF
:102FC000911D8F2D61E00E94911D8AE090E00E948A
:102FD000E01C8F2D0E94C41D892B11F410E00FC03E
:102FE000802F60E00E94911D8AE090E00E94E01C2A
:102FF0008F2D0E94C41D10E0892B09F411E0802F51
:1030000060E00E94251D802F60E00E94911D8F2DA1
:1030100060E00E94911D812F1F910F91FF900895F4
:10302000EF92FF920F931F937C0109E914E0C8010E
:103030006F2D70E04AE050E00E94011FC8016EE26F
:103040000E94401EB70184E0769567958A95E1F766
:103050006F707070C8014AE050E00E94011FC80103
:103060006EE20E94401E8FE0E822FF24C801B701F3
:103070004AE050E00E94011F1F910F91FF90EF90D6
:1030800008952F923F924F925F926F927F928F920C
:103090009F92AF92BF92CF92DF92EF92FF920F93E7
:1030A000DF93CF93CDB7DEB7A8970FB6F894DEBF06
:1030B0000FBECDBF7E010894E11CF11C80E1D70159
:1030C0001D928A95E9F789E994E064E471E00E9431
:1030D0008A1F0E94720E20E431EE4DE958E129A3C7
:1030E0003AA34BA35CA380EC91EDA8E9BBE18D8FE3
:1030F0009E8FAF8FB8A324EF31E040E050E0298FDE
:103100003A8F4B8F5C8F20E5822E23EC922EA12CE0
:10311000B12C80E491EEADE9B8E18D8B9E8BAF8B45
:10312000B88F44245524320100E022243324198A24
:103130001A8A1B8A1C8A0DC189E994E00E941A210F
:103140008434C9F0853434F48332C9F18C3209F007
:10315000CEC046C0833509F0CAC029A13AA14BA10F
:103160005CA1C901DA018D8B9E8BAF8BB88F442493
:1031700055243201EEC089E994E064E40E94401EC7
:1031800089E994E040E451EE6DE978E12AE030E02D
:103190000E94241F89E994E06CE20E94401E89E9A4
:1031A00094E040EC51ED68E97BE12AE030E00E94D8
:1031B000241F89E994E06CE20E945E1ECAC0198255
:1031C0001A821B821C821D821E821F82188619860B
:1031D0001A861B861C861D861E861F86188A3CC082
:1031E0000F5F043009F0B5C069817A818B819C81C1
:1031F00028EE33E040E050E00E94E72169A37AA383
:103200008BA39CA36D817E818F8198850E94E7218D
:103210006D8F7E8F8F8F98A329853A854B855C852E
:10322000298F3A8F4B8F5C8F6D857E858F8598892E
:1032300028EE33E040E050E00E94E7214B015C01C2
:1032400060323EE4730730E0830730E0930730F4E8
:103250008CE162E30E948A0300E07BC0603345E7B3
:10326000740740E0840740E0940718F48CE162E2C0
:10327000F1CF60345CE9750750E0850750E09507B1
:1032800018F48CE166E2E6CF80E5881683EC9806B8
:1032900080E0A80680E0B80618F48CE162E1DACF9D
:1032A00090E689169AEE990690E0A90690E0B90694
:1032B00018F48CE165E1CECFA0E78A16A1E19A0669
:1032C000A1E0AA06A0E0BA0618F48CE161E0C2CF42
:1032D000B0EA8B16B6E89B06B1E0AB06B0E0BB06E1
:1032E00018F48CE163E0B6CF8CE165E0B3CF805396
:1032F0008A3078F5C02EDD24CC0CDD1CCC0CDD1C16
:10330000E1E0F0E0EC0FFD1FCE0EDF1E282F33278B
:1033100027FD3095432F532F2DA33EA34FA358A72E
:10332000D6016D917D918D919C912AE030E040E035
:1033300050E00E94E7212DA13EA14FA158A5260FE4
:10334000371F481F591FD6012D933D934D935C9312
:10335000139789E994E00E94E020892B09F0ECCED4
:10336000411451046104710499F46D897E898F8937
:10337000988D0E941B0461E070E080E090E00E9464
:10338000BA1C22242A943324198A1A8A1B8A1C8A7A
:10339000298D3A8D4B8D5C8D421653066406750659
:1033A000D0F40E94AB0329893A894B895C89280FA4
:1033B000311D411D511D298B3A8B4B8B5C8B38166F
:1033C00008F4382E821508F4282E0894411C511C4C
:1033D000611C711C64C06D897E898F89988D28EE6F
:1033E00033E040E050E00E941A2289E994E0BA01FB
:1033F000A9012AE030E00E94F21E89E994E06CE223
:103400000E94401E89E994E0632D4AE050E00E944A
:10341000121F89E994E06CE20E94401E69897A8952
:103420008B899C89A30192010E941A2289E994E068
:10343000BA01A9012AE030E00E94F21E89E994E075
:103440006CE20E94401E89E994E0622D4AE050E05F
:103450000E94121F89E994E06CE20E945E1E8D8931
:103460009E89AF89B88D880D991DAA1DBB1D8D8BB6
:103470009E8BAF8BB88F2D8D3E8D4F8D58A1281709
:1034800039074A075B0740F489A19AA1ABA1BCA107
:103490008D8B9E8BAF8BB88F44245524320129A18C
:1034A0003AA14BA15CA1285E33404040504009F056
:1034B00050CFA8960FB6F894DEBF0FBECDBFCF9108
:1034C000DF910F91FF90EF90DF90CF90BF90AF9082
:1034D0009F908F907F906F905F904F903F902F9034
:1034E000089580E065E970E042E050E00E94C11B71
:1034F0000895DF93CF930F92CDB7DEB785E061E0FB
:103500000E94251D86E061E00E94251D0E945D0E3F
:1035100080E060E00E94251D81E061E00E94251DA1
:1035200089E994E040E052EC61E070E00E945920AB
:103530000E94460F0E94100889E994E061E571E05D
:103540000E94871F84E593E00E94101889E994E0A7
:1035500068E671E00E94871F89E994E065E070E009
:103560004AE050E00E94731F0E94711A78945E9A9C
:1035700083E063E10E94D517882329F05E985D9867
:103580000E944118FBCF89E062E10E94D517882391
:1035900029F40E94A400892B09F0EBC089E994E08A
:1035A00060E771E00E94871F60E070E080E090E0DB
:1035B0000E94890F882349F00E94771089E994E0DE
:1035C00069EA71E00E948A1F5D9A0E94801122C000
:1035D00080910003833229F080910A038B7F8093CE
:1035E0000A0380910A0381FF15C082FD13C064EFB6
:1035F00071E080E090E00E94890F882359F00E94DA
:10360000771089E994E069EA71E00E948A1F0E94BC
:1036100080115D9A8091FE02823239F5809100031B
:10362000833219F581E00E94B11280910A0382FF72
:1036300009C089E994E064EC71E00E948A1F0E944D
:10364000E80813C064E170E080E090E00E94BA1CDA
:1036500080E2BE016F5F7F4F41E021E00E946F0971
:10366000882319F481E08093830389E994E06FEC67
:1036700071E00E94871F80E00E948704109241033E
:1036800080E00E9495031092FF0390E0983158F477
:10369000292F2F5FE92FF0E0ED52FD4F878588231A
:1036A00011F0922FF3CF9093FF0383E08093D20227
:1036B0000E94720E80918303882311F00E94FD0AFC
:1036C00080910403883211F08A3239F489E994E058
:1036D00040E052EC61E070E02BC0893271F489E97E
:1036E00094E040EA56E861E070E00E945920809141
:1036F000C20080628093C20022C08091FB02887168
:10370000803169F04091D4025091D5026091D60287
:103710007091D7024A3051056105710538F489E985
:1037200094E040E855E260E070E002C089E994E08E
:103730000E94592004C089E994E00E941A2189E975
:1037400094E00E94E020892BB1F71092FD031092C3
:10375000FE03109281030E94941C609342037093B5
:10376000430380934403909345030F90CF91DF91DF
:1037700008950E9480118091FE02823209F02CCFC0
:1037800027CF823000F5E82FF0E0EE0FFF1FEC5F4F
:10379000FB4F71836083882319F08130A1F408C046
:1037A000809169008C7F842B80936900E89A08954A
:1037B00080916900440F551F440F551F837F842B50
:1037C00080936900E99A08951F920F920FB60F92A5
:1037D00011242F933F934F935F936F937F938F9316
:1037E0009F93AF93BF93EF93FF93809104049091C5
:1037F0000504892B29F0E0910404F0910504099552
:10380000FF91EF91BF91AF919F918F917F916F91B8
:103810005F914F913F912F910F900FBE0F901F908E
:1038200018951F920F920FB60F9211242F933F936A
:103830004F935F936F937F938F939F93AF93BF93B8
:10384000EF93FF938091060490910704892B29F050
:10385000E0910604F09107040995FF91EF91BF9163
:10386000AF919F918F917F916F915F914F913F9118
:103870002F910F900FBE0F901F9018951F920F92CF
:103880000FB60F9211242F933F938F939F93AF9373
:10389000BF9380910C0490910D04A0910E04B091FF
:1038A0000F04309110040196A11DB11D232F2D5F2F
:1038B0002D3720F02D570196A11DB11D2093100426
:1038C00080930C0490930D04A0930E04B0930F0406
:1038D0008091080490910904A0910A04B0910B040E
:1038E0000196A11DB11D8093080490930904A09333
:1038F0000A04B0930B04BF91AF919F918F913F91B8
:103900002F910F900FBE0F901F9018958FB7F894BE
:1039100020910C0430910D0440910E0450910F043D
:103920008FBFB901CA0108959FB7F8942091080488
:103930003091090440910A0450910B0486B5A89B6C
:1039400006C08F3F21F02F5F3F4F4F4F5F4F9FBF0C
:10395000542F432F322F2227280F311D411D511D77
:1039600082E0220F331F441F551F8A95D1F7B901FA
:10397000CA010895EF92FF920F931F93CF93DF93A5
:103980007B018C010E94941CEB010EC00E94941CD0
:103990006C1B7D0B685E7340C8F30894E108F10866
:1039A00001091109C851DC4FE114F10401051105A9
:1039B00069F7DF91CF911F910F91FF90EF900895DC
:1039C000019739F0880F991F880F991F0297019767
:1039D000F1F70895789484B5826084BD84B58160E0
:1039E00084BD85B5826085BD85B5816085BDEEE607
:1039F000F0E0808181608083E1E8F0E010828081E6
:103A000082608083808181608083E0E8F0E0808153
:103A100081608083E1EBF0E0808184608083E0EB73
:103A2000F0E0808181608083EAE7F0E0808184605B
:103A300080838081826080838081816080838081B7
:103A4000806880831092C1000895CF93DF93482F40
:103A500050E0CA0186569F4FFC0134914A575F4F90
:103A6000FA018491882369F190E0880F991FFC0185
:103A7000E859FF4FA591B491FC01EE58FF4FC59155
:103A8000D491662351F42FB7F8948C91932F90958D
:103A900089238C93888189230BC0623061F42FB70E
:103AA000F8948C91932F909589238C938881832B04
:103AB00088832FBF06C09FB7F8948C91832B8C937B
:103AC0009FBFDF91CF910895833071F0843028F447
:103AD0008130A1F0823021F514C08630B1F08730FA
:103AE000D1F08430E9F404C0809180008F7703C066
:103AF000809180008F7D80938000089584B58F77BA
:103B000002C084B58F7D84BD08958091B0008F7709
:103B10008093B00008958091B0008F7D8093B000B5
:103B20000895FF920F931F93F62E482F50E0CA017D
:103B300082559F4FFC012491CA0186569F4FFC017C
:103B400014914A575F4FFA0104910023C9F02223D0
:103B500019F0822F0E94641DE02FF0E0EE0FFF1F8E
:103B6000EE58FF4FA591B4919FB7F894FF2021F430
:103B70008C911095812302C08C91812B8C939FBFD7
:103B80001F910F91FF9008950F931F93482F50E0BE
:103B9000CA0182559F4FFC012491CA0186569F4F4E
:103BA000FC0104914A575F4FFA011491112319F453
:103BB00020E030E015C0222319F0822F0E94641DFE
:103BC000812F90E0880F991F84589F4FFC01A59189
:103BD000B4918C9120E030E0802311F021E030E0BE
:103BE000C9011F910F910895982F8E3008F09E50B3
:103BF0009770809199028295880F880F807C892B1D
:103C000080937C0080917A00806480937A00809118
:103C10007A0086FDFCCF2091780040917900942FA6
:103C200080E030E0282B392BC9010895CF92DF9234
:103C3000EF92FF920F931F93CF93DF937C016B0161
:103C40008A01C0E0D0E00FC0D6016D916D01D701AF
:103C5000ED91FC910190F081E02DC7010995C80F0D
:103C6000D91F015010400115110571F7CE01DF91E8
:103C7000CF911F910F91FF90EF90DF90CF9008951B
:103C8000DC01ED91FC910190F081E02D0995089502
:103C9000EF92FF920F931F938C016DE00E94401EE4
:103CA0007C01C8016AE00E94401E9C012E0D3F1D50
:103CB000C9011F910F91FF90EF900895EF92FF922D
:103CC0000F931F937C010E94401E8C01C7010E942C
:103CD000481E9C01200F311FC9011F910F91FF90B9
:103CE000EF900895CF93DF93EC016115710519F4FE
:103CF00020E030E00FC0DB010D900020E9F71197C4
:103D0000A61BB70BE881F9810280F381E02DAD019C
:103D100009959C01C901DF91CF9108954F925F925F
:103D20007F928F929F92AF92BF92CF92DF92EF924B
:103D3000FF920F931F93DF93CF93CDB7DEB7A19779
:103D40000FB6F894DEBF0FBECDBF2C01742ECB0191
:103D5000223008F42AE019A231E2C32ED12CCC0E75
:103D6000DD1E822E9924AA24BB24672D752FA50160
:103D700094010E941A2279018A01C801B701A501A4
:103D800094010E94E721472D461B0894C108D108E1
:103D90004A3014F4405D01C0495CF6014083E114EF
:103DA000F1040105110521F07E2C5F2DC801DDCF46
:103DB000C201B6010E94721EA1960FB6F894DEBF32
:103DC0000FBECDBFCF91DF911F910F91FF90EF906C
:103DD000DF90CF90BF90AF909F908F907F905F903B
:103DE0004F900895DC012115310541F4ED91FC91CE
:103DF0000190F081E02D642F099508950E948E1E98
:103E00000895EF92FF920F931F939A017B0100E0B8
:103E100010E0B801A7010E94F21E1F910F91FF90C0
:103E2000EF900895EF92FF920F931F939A01E62E61
:103E3000FF2400E010E0B801A7010E94F21E1F91CC
:103E40000F91FF90EF900895CF92DF92EF92FF9243
:103E50000F931F93CF93DF93EC016A017B01211530
:103E6000310541F4E881F9810190F081E02D642F62
:103E700009951BC02A303105B1F477FF13C06DE2FC
:103E80000E94401E8C0144275527BA014C195D0938
:103E90006E097F09CE012AE00E948E1E9C01200F30
:103EA000311F04C02AE00E948E1E9C01C901DF91CF
:103EB000CF911F910F91FF90EF90DF90CF900895D9
:103EC000EF92FF920F931F937B019A010027F7FC5B
:103ED0000095102FB801A7010E94241F1F910F9178
:103EE000FF90EF900895EF92FF920F931F937C0144
:103EF0000E94601F8C01C7010E94481E9C01200F78
:103F0000311FC9011F910F91FF90EF9008950E94FA
:103F1000721E0895EF92FF920F931F937C010E94EF
:103F2000871F8C01C7010E94481E9C01200F311F72
:103F3000C9011F910F91FF90EF90089508951F926E
:103F40000F920FB60F9211242F933F934F938F939D
:103F50009F93EF93FF938091C00082FD1DC040911D
:103F6000C60020915104309152042F5F3F4F2F73B0
:103F7000307080915304909154042817390771F0E0
:103F8000E0915104F0915204EF5EFB4F4083309377
:103F900052042093510402C08091C600FF91EF911A
:103FA0009F918F914F913F912F910F900FBE0F9046
:103FB0001F9018951F920F920FB60F9211242F93F6
:103FC0003F938F939F93EF93FF93209195043091AC
:103FD000960480919704909198042817390731F43A
:103FE0008091C1008F7D8093C10014C0E09197043F
:103FF000F0919804EB5AFB4F2081809197049091A7
:10400000980401968F73907090939804809397040E
:104010002093C600FF91EF919F918F913F912F9137
:104020000F900FBE0F901F9018958F929F92AF9296
:10403000BF92CF92DF92EF92FF920F931F93DF9385
:10404000CF93CDB7DEB7FC011382128288EE93E0E6
:10405000A0E0B0E084839583A683B78386EC92E0EA
:10406000918380837587648757874687318B208B40
:10407000138B028BF58AE48AD78AC68AB18EA08E0A
:10408000938E828E8F85848F8889858F8989868F8C
:104090008A89878F8B8980A3CF91DF911F910F91A0
:1040A000FF90EF90DF90CF90BF90AF909F908F9058
:1040B0000895AF92BF92DF92EF92FF920F931F93FA
:1040C000CF93DF93EC017A018B01DD24403081EE48
:1040D000580780E0680780E0780711F0DD24D3946A
:1040E00091E0A92EB12CEC89FD89DD2069F0C50194
:1040F00008A002C0880F991F0A94E2F7808360E04D
:1041000079E08DE390E005C0108260E874E88EE10C
:1041100090E0A80197010E941A22215030404040AF
:104120005040569547953795279580E120303807C0
:1041300020F0DD2011F0DD24D6CFE889F989308325
:10414000EA89FB89208319A2EE89FF89408121E059
:1041500030E0C9010C8C02C0880F991F0A94E2F765
:10416000482B4083EE89FF894081C9010D8C02C034
:10417000880F991F0A94E2F7482B4083EE89FF8944
:104180004081C9010E8C02C0880F991F0A94E2F782
:10419000482B4083EE89FF8980810F8C02C0220F5B
:1041A000331F0A94E2F7209528232083DF91CF91D3
:1041B0001F910F91FF90EF90DF90BF90AF90089507
:1041C000DC011C96ED91FC911D97E05CFF4F219165
:1041D000319180819181281B390B2F733070C90177
:1041E000089589E994E00E94E020892B11F00E9453
:1041F0009E1F0895DC011C96ED91FC911D97E05CDB
:10420000FF4F20813181E054F040DF01AE5BBF4FB2
:104210008D919C9111972817390719F42FEF3FEFD3
:1042200007C08D919C91E80FF91F8081282F30E005
:10423000C9010895DC011C96ED91FC911D97E05C8D
:10424000FF4F20813181E054F040DF01AE5BBF4F72
:104250008D919C9111972817390719F42FEF3FEF93
:1042600010C08D919C911197E80FF91F20818D91BD
:104270009C91119701968F73907011969C938E93D9
:1042800030E0C9010895DC0191968C9191978823C3
:1042900039F05496ED91FC915597808186FFF9CFC6
:1042A00091961C920895CF93DF93EC01EE85FF85E4
:1042B000E05CFF4F20813181E054F0402F5F3F4FA1
:1042C0002F733070DF01AE5BBF4F8D919C911197C2
:1042D00028173907D1F3E05CFF4F80819181E054CA
:1042E000F040E80FF91F6083EE85FF85E05CFF4F2B
:1042F00031832083EE89FF89208181E090E00F8C5B
:1043000002C0880F991F0A94E2F7282B208381E0CE
:1043100089A3EC89FD8980818064808381E090E0BD
:10432000DF91CF9108958F929F92AF92BF92CF92DB
:10433000DF92EF92FF920F931F9300D000D00F9265
:10434000EDB7FEB7319684E0ADB7BEB711968C934A
:1043500083E0818387E0828385E0838381E08483B7
:1043600089E994E061E174E045E554E025EC30E052
:1043700004EC10E0B0ECEB2EF12CA1ECCA2ED12C09
:10438000F2ECAF2EB12CE6EC8E2E912C0E94152073
:104390000F900F900F900F900F901F910F91FF9023
:1043A000EF90DF90CF90BF90AF909F908F90089547
:1043B000CF93DF930E94EA1C0E94791AC1EFD0E2EA
:1043C0000E94C4132097E1F30E94F120F9CF629F6D
:1043D000D001739FF001829FE00DF11D649FE00DFD
:1043E000F11D929FF00D839FF00D749FF00D659F5E
:1043F000F00D9927729FB00DE11DF91F639FB00D5D
:10440000E11DF91FBD01CF0111240895AA1BBB1B9B
:1044100051E107C0AA1FBB1FA617B70710F0A61BC4
:10442000B70B881F991F5A95A9F780959095BC01E5
:10443000CD010895A1E21A2EAA1BBB1BFD010DC0E0
:10444000AA1FBB1FEE1FFF1FA217B307E407F50744
:1044500020F0A21BB30BE40BF50B661F771F881F20
:10446000991F1A9469F760957095809590959B01B6
:10447000AC01BD01CF01089597FB092E05260ED092
:1044800057FD04D0D7DF0AD0001C38F45095409572
:10449000309521953F4F4F4F5F4F0895F6F7909518
:1044A0008095709561957F4F8F4F9F4F0895EE0FC8
:0E44B000FF1F0590F491E02D0994F894FFCFC2
:1044BE0054582074696D656F757421005258636F7E
:1044CE006E66206C6F616465640057616974696E15
:1044DE00672062696E640A00476F7420706B740AFD
:1044EE00006461746120676F6F640A00525820681F
:1044FE00616E67007363616E6E6572206D6F6465C9
:10450E00004F70656E4C52536E6720525820737474
:10451E00617274696E672000206F6E20485720000C
:10452E00454550524F4D2064617461206E6F74206A
:10453E0076616C6964206F722062696E64206A75A0
:10454E006D70706572207365742C20666F7263696E
:10455E006E672062696E640A00536176656420623C
:10456E00696E64206461746120746F2045455052F9
:10457E004F4D0A004920616D20736C6176650045D0
:10458E006E746572696E67206E6F726D616C206DF0
:10459E006F646500002001220126022102270323F9
:1045AE00032604260526052B06240725072807299A
:1045BE00072AC01200001A400AA1204EA5001B1E99
:1045CE0027522C23308025000005400AA1204EA53D
:1045DE000020244EA52C2330004B000006400AD0AC
:1045EE00009D49007B289D492C233000E1000005E9
:1045FE00400A4501D7DC03B81E0EBF00232E48E843
:10460E0001008A400A6001555502AD1E20000023AC
:10461E00C88025000005400AA1204EA50020244E8A
:10462E00A52C23300002000200020002000200024C
:10463E00000200020002000200020002000200025C
:10464E00000200028813409C0801091203130E0F8A
:10465E000001020000001000000008002000000110
:10466E000000020000000100000200070B0C1011F8
:10467E001500000000005321161EE0201A21FA201A
:02468E004321C6
:00000001FF
